:1000000077EF07F0FFFFFFFF6E0E0001CB6F6F0E63
:10001000CC6F6E0ECD6F2D0ECE6F6C0ECF6F6F0E40
:10002000D06F6E0ED16F670ED26F200ED36F700E31
:10003000D46F720ED56F690ED66F6E0ED76F740EB9
:10004000D86F660ED96FDA6B6E0EDB6F6F0EDC6FDA
:100050006E0EDD6F2D0EDE6F660EDF6F6C0EE06FC5
:100060006F0EE16F610EE26F740EE36F200EE46FAE
:10007000700EE56F720EE66F690EE76F6E0EE86F39
:10008000740EE96F660EEA6FEB6B280EEC6F6E0E66
:10009000ED6F750EEE6F6C0EEF6F6C0EF06F290E3C
:1000A000F16FF26BFA6BFB6BF86BF96B0001C6C07A
:1000B00000F0C7C001F0C8C002F0010EC627000E54
:1000C000C723C82300C0F6FF01C0F7FF02C0F8FF36
:1000D0000900F5CF00F000C0F5F00052D8B472EF7F
:1000E00007F0F551250A0BE0C4C0E1FFC5C0E2FFEF
:1000F000F5C0E6FFC44BC52BFA4BFB2BD7D7F66BED
:10010000F76BF86BF96B000128D00001F887010E3E
:10011000C627000EC723C8235ED00001F881010E58
:10012000C627000EC723C82356D00001F883010E4E
:10013000C627000EC723C8234ED00001F987010E41
:10014000C627000EC723C82346D00001F885010E3C
:10015000C627000EC723C8233ED0C6C0F6FFC7C0BF
:10016000F7FFC8C0F8FF0900F5CF00F10101005109
:100170002D0ACBE0C6C0F6FFC7C0F7FFC8C0F8FF26
:100180000900F5CF00F10051200AC7E0C6C0F6FF14
:10019000C7C0F7FFC8C0F8FF0900F5CF00F1005154
:1001A0002B0AC3E0C6C0F6FFC7C0F7FFC8C0F8FF00
:1001B0000900F5CF00F10051230ABFE0C6C0F6FFE9
:1001C000C7C0F7FFC8C0F8FF0900F5CF00F1005124
:1001D000300ABBE002D0010196D70001F8B3F891D4
:1001E000F8B7F895C6C0F6FFC7C0F7FFC8C0F8FF5C
:1001F0000900F5CF00F0000E016E00C003F11CEC09
:100200000EF0005239E00001F66BF76BF6C000F01B
:10021000F7C001F00A0E046E000E056E87EC0CF0BC
:10022000C6C0F6FFC7C0F7FFC8C0F8FF0900F5CF8A
:1002300000F10101005100240001F66F000E0120C1
:10024000F76F300EF65F000EF75B010EC627000E4B
:10025000C723C823C6C0F6FFC7C0F7FFC8C0F8FF52
:100260000900F5CF00F0000E016E00C003F11CEC98
:100270000EF00052CBE137D0C6C0F6FFC7C0F7FF83
:10028000C8C0F8FF0900F5CF00F1010100512A0AAA
:100290002AE1C9C0E9FFCAC0EAFFEECF00F0EECF05
:1002A00001F000C0E9FF01C0EAFFEECFF6F0EECFAB
:1002B000F7F0C9C0E9FFCAC0EAFFEECF00F0EECF09
:1002C00001F0020E0026000E0122C9C0E1FFCAC0E3
:1002D000E2FF00C0E6FF01C0E6FF010E0001C627F5
:1002E000000EC723C8230001C6C0F6FFC7C0F7FF32
:1002F000C8C0F8FF0900F5CF00F1010100512E0A36
:10030000D8A479D0010E0001C627000EC723C82348
:10031000C6C0F6FFC7C0F7FFC8C0F8FF0900F5CF99
:1003200000F1010100512A0A2BE1C9C0E9FFCAC04E
:10033000EAFFEECF00F0EECF01F000C0E9FF01C010
:10034000EAFFEECFF3F0EECFF4F0C9C0E9FFCAC088
:10035000EAFFEECF00F0EECF01F0020E0026000E15
:100360000122C9C0E1FFCAC0E2FF00C0E6FF01C030
:10037000E6FF010E0001C627000EC723C82339D0AF
:100380000001F36BF46BC6C0F6FFC7C0F7FFC8C02F
:10039000F8FF0900F5CF00F0000E016E00C003F178
:1003A0001CEC0EF0005225E0F3C000F0F4C001F0A8
:1003B0000A0E046E000E056E87EC0CF0C6C0F6FF48
:1003C000C7C0F7FFC8C0F8FF0900F5CF00F1010171
:1003D000005100240001F36F000E0120F46F300E75
:1003E000F35F000EF45B010EC627000EC723C8237F
:1003F000CAD7000103D00001F36BF46B0001C6C043
:1004000000F0C7C001F0C8C002F0010EC627000E00
:10041000C723C82300C0F6FF01C0F7FF02C0F8FFE2
:100420000900F5CFF5F002D1FAC000F0FBC001F0F1
:100430001200CB0EFC6F000EFD6FF36BF46BFF0E22
:10044000F86FFF0EF96F31D0DB0EFC6F000EFD6F01
:10045000F36BF46B2AD0F88D24D123D1F88BF88F6D
:1004600020D1C9C0E9FFCAC0EAFFEECF00F0EECF4D
:1004700001F000C0E9FF01C0EAFFEECFFCF0EECFD3
:10048000FDF0C9C0E9FFCAC0EAFFEECF00F0EECF31
:1004900001F0020E0026000E0122C9C0E1FFCAC011
:1004A000E2FF00C0E6FF01C0E6FF000EFD1902E119
:1004B000000EFC1904E1EC0EFC6F000EFD6F000154
:1004C000FE6BFF6BFE51FC25E96EFF51FD21EA6ECC
:1004D000EECF00F0005203E0FE4BFF2BF3D7F351B9
:1004E000F4110AE0FF51F45D02E1FE51F35D04E214
:1004F000F3C0FEF0F4C0FFF00001F751FF5D02E130
:10050000F651FE5D05E2FE51F65FFF51F75B03D049
:100510000001F66BF76BF8B716D0F6C000F0F7C025
:1005200001F0010EF65F000EF75B005001100BE0CA
:10053000C4C0E1FFC5C0E2FF200EE66EC44BC52B70
:10054000FA4BFB2BEAD7FEC000F0FFC001F0010E12
:10055000FE5F000EFF5B0050011013E0FCC0E9FFDE
:10056000FDC0EAFFEECF00F0C4C0E1FFC5C0E2FF6E
:1005700000C0E6FFC44BC52BFC4BFD2BFA4BFB2BFD
:10058000E2D7F8A716D0F6C000F0F7C001F0010ED0
:10059000F65F000EF75B005001100BE0C4C0E1FFF6
:1005A000C5C0E2FF200EE66EC44BC52BFA4BFB2BF9
:1005B000EAD7F951FF0A02E1FF0EF81905E1FAC086
:1005C00000F0FBC001F01200000170D5C9C0E9FFC6
:1005D000CAC0EAFFEECF00F0EECF01F000C0E9FFA5
:1005E00001C0EAFFEECFF5F0C9C0E9FFCAC0EAFFDB
:1005F000EECF00F0EECF01F0020E0026000E012239
:10060000C9C0E1FFCAC0E2FF00C0E6FF01C0E6FFCB
:10061000F50EFC6F000EFD6F010EFE6F000EFF6FFA
:100620005ED7C00EF813000EF9133BD0F551000A47
:10063000D8B4FAD6F5516C0AD8B4FBD6F551450AB0
:10064000D8B402D7F551660AD8B4FED6F551650A7A
:10065000D8B4FAD6F551670AD8B4F6D6F5516F0A70
:10066000D8B4F9D6F551640AD8B4F7D6F551690A69
:10067000D8B4F3D6F551700AD8B4F0D6F551580A6B
:10068000D8B4ECD6F551780AD8B4E9D6F551730A46
:10069000D8B4E7D6F551630A99E0F551750AC1E07F
:1006A000B7D70001C00EF8150101006FF9C001F1C4
:1006B000000E0117000E011902E1000E00193FE1C2
:1006C000C9C0E9FFCAC0EAFFEECF00F0EECF01F0EB
:1006D00000C0E9FF01C0EAFFEECFFCF0EECFFDF075
:1006E000C9C0E9FFCAC0EAFFEECF00F0EECF01F0CB
:1006F000020E0026000E0122C9C0E1FFCAC0E2FFBF
:1007000000C0E6FF01C0E6FF800E0001FD19006E8B
:10071000800E005C02E1000EFC5D0FE2030EF81398
:10072000000EF913FC510008006EFDC001F0E86AEC
:10073000015600C0FCF001C0FDF0000125D0000111
:10074000C9C0E9FFCAC0EAFFEECF00F0EECF01F06A
:1007500000C0E9FF01C0EAFFEECFFCF0EECFFDF0F4
:10076000C9C0E9FFCAC0EAFFEECF00F0EECF01F04A
:10077000020E0026000E0122C9C0E1FFCAC0E2FF3E
:1007800000C0E6FF01C0E6FF0001000EF41902E11F
:10079000000EF31908E1000EFD1902E1000EFC192C
:1007A00002E1F34BF42B0001C00EF815006E00C0FF
:1007B00002F1A9D000010001010EF56FF551050A03
:1007C00030E0010E046EF5C000F0000E016E026E06
:1007D000036E0450000107E0003600900136023637
:1007E0000336FF0FF7D7600E00261C0E0122000E05
:1007F000022200C0F6FF01C0F7FF02C0F8FF0900A7
:10080000F5CF00F10900F5CF01F10101015100011F
:10081000FD5D04E1010100510001FC5D02E3F52BE7
:10082000CDD700017FD00001010EF56FF551040A0C
:1008300030E0010E046EF5C000F0000E016E026E95
:10084000036E0450000107E00036009001360236C6
:100850000336FF0FF7D76A0E00261C0E0122000E8A
:10086000022200C0F6FF01C0F7FF02C0F8FF090036
:10087000F5CF00F10900F5CF01F1010101510001AF
:10088000FD5D04E1010100510001FC5D02E3F52B77
:10089000CDD7000147D00001010EF56FF551060AD2
:1008A00030E0010E046EF5C000F0000E016E026E25
:1008B000036E0450000107E0003600900136023656
:1008C0000336FF0FF7D7720E00261C0E0122000E12
:1008D000022200C0F6FF01C0F7FF02C0F8FF0900C6
:1008E000F5CF00F10900F5CF01F10101015100013F
:1008F000FD5D04E1010100510001FC5D02E3F52B07
:10090000CDD700010FD001010251000AD8B452D74F
:100910000251C00AD8B44ED70251800A84E0025175
:10092000400AB9E0800E006E800E0001F419005CF0
:1009300002E1F351F55D03E2F3C0F5F00ED00001E2
:10094000800EF419006E800E005C02E1F551F35D3B
:1009500004E2F5C0F3F0000EF46F00010001F6515F
:10096000F7110EE0030EF815006EF9C001F0000E4D
:1009700001160050011004E0010EF65F000EF75B57
:10098000800EF419006E800EF719005C02E1F6513A
:10099000F35D05E2F351F65FF451F75B03D000011C
:1009A000F66BF76BC40EF8150101006F0001F951E9
:1009B000080B0101016F0151080A02E1400E001904
:1009C00009E10001F651F71104E0010EF65F000E97
:1009D000F75B22D00001C00EF8150101006F000185
:1009E000F951080B0101016F0151080A02E1800E63
:1009F000001912E1800E006E800E0001F719005CF4
:100A000002E1F651020805E2020EF65F000EF75B06
:100A100003D00001F66BF76B00010001F8A572D05E
:100A2000F8A31AD0010EF815006EF9C001F0000EFF
:100A300001160050011003E02D0E006E02D02B0EA7
:100A4000006EC4C0E1FFC5C0E2FF00C0E6FFC44BBA
:100A5000C52BFA4BFB2B40D0010EF815006EF9C0E8
:100A600001F0000E0116005001100BE0C4C0E1FFC0
:100A7000C5C0E2FF200EE66EC44BC52BFA4BFB2B24
:100A80002BD0C00EF8150101006F0001F951080BC1
:100A90000101016F0151080A02E1800E00191CE1F9
:100AA000C4C0E1FFC5C0E2FF300EE66E0001C44BDA
:100AB000C52BFA4BFB2BF8AB03D0580E006E02D0BF
:100AC000780E006EC4C0E1FFC5C0E2FF00C0E6FFC3
:100AD000C44BC52BFA4BFB2B0001F651F71111E06B
:100AE000C4C0E1FFC5C0E2FF300EE66EC44BC52BAB
:100AF000FA4BFB2B010EF65F000EF75BF651F71178
:100B0000EFE18DD0F651F71113E0F8B711D0C4C062
:100B1000E1FFC5C0E2FF200EE66EC44BC52BFA4BC9
:100B2000FB2B010EF65F000EF75BF651F711EFE1BC
:100B3000F8A31AD0010EF815006EF9C001F0000EEE
:100B400001160050011003E02D0E006E02D02B0E96
:100B5000006EC4C0E1FFC5C0E2FF00C0E6FFC44BA9
:100B6000C52BFA4BFB2B14D0010EF815006EF9C003
:100B700001F0000E0116005001100AE0C4C0E1FFB0
:100B8000C5C0E2FF200EE66EC44BC52BFA4BFB2B13
:100B9000C00EF8150101006F0001F951080B0101A9
:100BA000016F0151080A02E1400E00190CE1C4C0B6
:100BB000E1FFC5C0E2FF300EE66E0001C44BC52B5D
:100BC000FA4BFB2B2CD00001C00EF8150101006F71
:100BD0000001F951080B0101016F0151080A02E1FE
:100BE000800E00191CE1C4C0E1FFC5C0E2FF300E59
:100BF000E66E0001C44BC52BFA4BFB2BF8AB03D0C0
:100C0000580E006E02D0780E006EC4C0E1FFC5C061
:100C1000E2FF00C0E6FFC44BC52BFA4BFB2B0001E3
:100C20000001800E006E800EF419005C02E1F351A9
:100C3000F55D0BE2C4C0E1FFC5C0E2FF300EE66E19
:100C4000C44BC52BFA4BFB2BEAD70001F3C000F0D5
:100C5000F4C001F0010EF35F000EF45B00500110D0
:100C6000D8B421D1C00EF815006E00C000F1FFD03D
:100C700000010001010E046EF3C000F0F4C001F0A9
:100C8000000EF4BFFF0E026E036E0450000107E079
:100C900000360090013602360336FF0FF7D7000109
:100CA000600E00261C0E0122000E022200C0F6FF7C
:100CB00001C0F7FF02C0F8FF0900F5CF04F00900FA
:100CC000F5CF05F0FCC000F0FDC001F0D2EC0DF056
:100CD0000A0E046E000E056ED2EC0DF008C000F096
:100CE00009C001F0300E0024F56FD1D00001F8AB3F
:100CF00044D0010E046EF3C000F0F4C001F0000E09
:100D0000F4BFFF0E026E036E0450000107E00036D0
:100D10000090013602360336FF0FF7D700016A0E46
:100D200000261C0E0122000E022200C0F6FF01C0A8
:100D3000F7FF02C0F8FF0900F5CF04F00900F5CF76
:100D400005F0FCC000F0FDC001F0D2EC0DF00F0E7C
:100D50000016000E0116000E026E7E0E00261C0EFE
:100D60000122000E022200C0F6FF01C0F7FF02C000
:100D7000F8FF0900F5CFF5F043D0010E046EF3C083
:100D800000F0F4C001F0000EF4BFFF0E026E036E1F
:100D90000450000107E000360090013602360336A9
:100DA000FF0FF7D700016A0E00261C0E0122000E6D
:100DB000022200C0F6FF01C0F7FF02C0F8FF0900E1
:100DC000F5CF04F00900F5CF05F0FCC000F0FDC040
:100DD00001F0D2EC0DF00F0E0016000E0116000E01
:100DE000026E900E00261C0E0122000E022200C090
:100DF000F6FF01C0F7FF02C0F8FF0900F5CFF5F0DC
:100E0000000145D00001010E046EF3C000F0F4C0F3
:100E100001F0000EF4BFFF0E026E036E04500001DD
:100E200007E000360090013602360336FF0FF7D791
:100E30000001720E00261C0E0122000E022200C0CC
:100E4000F6FF01C0F7FF02C0F8FF0900F5CF04F07C
:100E50000900F5CF05F0FCC000F0FDC001F0D2ECB8
:100E60000DF0070E0014F56F300EF52710D00101BC
:100E70000051000AD8B4FCD60051C00AD8B4F8D644
:100E80000051800AD8B432D70051400ABBE0C4C038
:100E9000E1FFC5C0E2FFF5C0E6FF0001C44BC52B72
:100EA000FA4BFB2BD2D6F8A71AD0800E006E800E1C
:100EB000F719005C02E1F651000811E2C4C0E1FF3D
:100EC000C5C0E2FF200EE66EC44BC52BFA4BFB2BD0
:100ED000010EF65F000EF75BF651F711EFE100012E
:100EE00056EF00F0FAC000F0FBC001F01200500E07
:100EF000506E490E516E430E526E200E536E500EC0
:100F0000546E720E556E6F0E566E6A0E576E650EEB
:100F1000586E630E596E740E5A6E200E5B6E420E42
:100F20005C6E6F0E5D6E610E5E6E720E5F6E640EB5
:100F30000001606F616B500E626F490E636F430E6C
:100F4000646F310E656F380E666F460E676F340E34
:100F5000686F350E696F380E6A6F200E6B6F380E32
:100F60006C6F4D0E6D6F480E6E6F7A0E6F6F706BFB
:100F7000500E716F490E726F430E736F310E746FA6
:100F8000380E756F460E766F340E776F350E786FAC
:100F9000380E796F300E7A6F7B6B500E7C6F490E76
:100FA0007D6F430E7E6F310E7F6F360E806F460E63
:100FB000816F380E826F380E836F370E846F856BAA
:100FC000430E866F680E876F610E886F6E0E896F95
:100FD0006E0E8A6F650E8B6F6C0E8C6F310E8D6F7F
:100FE0003D0E8E6F300E8F6F2E0E906F300E916F04
:100FF000300E926F380E936F380E946F320E956FDD
:10100000370E966F560E976F986B430E996F680E5A
:101010009A6F610E9B6F6E0E9C6F6E0E9D6F650ECC
:101020009E6F6C0E9F6F320EA06F3D0EA16F310E42
:10103000A26F2E0EA36F320EA46F370EA56F320E65
:10104000A66F360EA76F330EA86F370EA96F560E18
:10105000AA6FAB6B500EAC6F490EAD6F430EAE6F07
:10106000200EAF6F740EB06F650EB16F720EB26F5F
:101070006D0EB36F690EB46F6E0EB56F610EB66F05
:101080006C0EB76FB86B810EB96F0F0EBA6F030E8F
:10109000BB6F020EBC6F040EBD6F050EBE6F070E58
:1010A000BF6F060EC06F830EC16F0F0EC26F05ECCF
:1010B00009F00001B96BF7EC0BF07A0E0001B96F83
:1010C0001D0EBA6F000EBB6F94EC0BF092EC0DF09E
:1010D00092EC0DF00001B96BF7EC0BF07A0E000109
:1010E000B96F210EBA6F000EBB6F94EC0BF092EC4F
:1010F0000DF092EC0DF07A0E0001B96F250EBA6F6B
:10110000000EBB6F050EBC6F080EBD6F200EBE6FCC
:10111000000EBF6F0DEC0EF00001B96BF7EC0BF099
:10112000500E0001B96F000EBA6FBB6BBC6B010EA5
:10113000BD6F6DEC0DF0620E0001B96F000EBA6F5D
:10114000BB6B010EBC6F010EBD6F6DEC0DF0710E2F
:101150000001B96F000EBA6FBB6B020EBC6F010EBF
:10116000BD6F6DEC0DF07C0E0001B96F000EBA6F13
:10117000BB6B030EBC6F010EBD6F6DEC0DF0860EE8
:101180000001B96F000EBA6FBB6B040EBC6F010E8D
:10119000BD6F6DEC0DF0990E0001B96F000EBA6FC6
:1011A000BB6B050EBC6F010EBD6F6DEC0DF0AC0E90
:1011B0000001B96F000EBA6FBB6B060EBC6F010E5B
:1011C000BD6F6DEC0DF0300E0001B96F000EBA6FFF
:1011D000640EBB6F270EBC6F000EBD6FFF0EBE6F9F
:1011E000FF0EBF6F47EC0DF0300EB96F000EBA6FF7
:1011F000BB6B070EBC6F010EBD6F6DEC0DF092EC7A
:101200000DF092EC0DF055D7FFD7C1C01BF0C2C056
:101210001CF0B9C015F0BAC016F0266AFF0E256E94
:10122000BBC001F0010E006E015004E000360090DA
:10123000FF0FFBD700C01DF0001C1F6EBCC001F0EB
:10124000010E006E015004E000360090FF0FFBD746
:1012500000C020F0001C1E6EBDC001F0010E006E2B
:10126000015004E000360090FF0FFBD700C021F0D2
:10127000001C196EBEC001F0010E006E015004E0AA
:1012800000360090FF0FFBD700C022F0001C1A6E42
:10129000BFC001F0010E006E015004E00036009066
:1012A000FF0FFBD700C02DF0001C2E6EC0C001F058
:1012B000010E006E015004E000360090FF0FFBD7D6
:1012C00000C017F0001C186E120E0001C125016E3F
:1012D000000EC221026E01C023F002C024F001C042
:1012E000E9FF02C0EAFFEECF00F0000E001601C0D9
:1012F000E1FF02C0E2FF00C0E6FF120E1524016EFE
:10130000000E1620026E01C023F002C024F001C0BE
:10131000E9FF02C0EAFFEECF00F01F50001601C047
:10132000E1FF02C0E2FF00C0E6FF23C0E9FF24C0E6
:10133000EAFFEECF00F01E50001623C0E1FF24C0EC
:10134000E2FF00C0E6FF23C0E9FF24C0EAFFEECFC2
:1013500000F01950001623C0E1FF24C0E2FF00C0D6
:10136000E6FF23C0E9FF24C0EAFFEECF00F01A50E9
:10137000001623C0E1FF24C0E2FF00C0E6FF23C047
:10138000E9FF24C0EAFFEECF00F02E50001623C084
:10139000E1FF24C0E2FF00C0E6FF23C0E9FF24C054
:1013A000EAFFEECF00F01850001623C0E1FF24C082
:1013B000E2FF00C0E6FF15C0E9FF16C0EAFFEECF6E
:1013C00000F02D50001215C0E1FF16C0E2FF00C072
:1013D000E6FF15C0E9FF16C0EAFFEECF00F0195096
:1013E000001615C0E1FF16C0E2FF00C0E6FF15C001
:1013F000E9FF16C0EAFFEECF00F01A50001615C044
:10140000E1FF16C0E2FF00C0E6FF15C0E9FF16C00D
:10141000EAFFEECF00F01F50001615C0E1FF16C026
:10142000E2FF00C0E6FF15C0E9FF16C0EAFFEECFFD
:1014300000F02050001215C0E1FF16C0E2FF00C00E
:10144000E6FF1BC0E1FF1CC0E2FF3F0EE66EB3ECFF
:101450000DF01BC0E1FF1CC0E2FFC00EE66EB3EC56
:101460000DF015C0E9FF16C0EAFFEECF00F01D50E9
:10147000001215C0E1FF16C0E2FF00C0E6FF15C074
:10148000E9FF16C0EAFFEECF00F01E50001615C0AF
:10149000E1FF16C0E2FF00C0E6FF1BC0E1FF1CC079
:1014A000E2FF3F0EE66EB3EC0DF01BC0E1FF1CC087
:1014B000E2FFC00EE66EB3EC0DF0050E296E070ECE
:1014C0002F6EA20E2A6E1C0E2B6E000E2C6E300E8E
:1014D000276E000E286E2FEC0EF012002750000130
:1014E000C45D006E28C001F0E86A015629C004F00E
:1014F000000E056E1EEC0DF000C0CCF001C0CDF06A
:10150000C5C003F1EEEC0CF0C6C003F1F0EC0DF039
:101510000001C86B2950C85D59E2C5C003F145EC14
:101520000CF0C6C003F1F0EC0DF0C5C003F1EEEC19
:101530000CF011EC0BF000C0C9F011EC0BF000C086
:10154000C9F0C5C003F145EC0CF0C6C003F1F0ECE6
:101550000DF0C5C003F1EEEC0CF00001CC512A24D3
:10156000006ECD512B20016E000ECDBFFF0E2C2042
:10157000026E000ECDBFFF0E00C0F6FF01C0F7FFE8
:1015800002C0F8FF0900F5CF00F000C0CAF0CC4B54
:10159000CD2B001CCB6F09D0CBC0C9F00FD0CAC077
:1015A000C9F00CD0CA51C91B09D0C751000AF4E0D8
:1015B000C751010AF4E0C751020AF4E0C9C003F1BF
:1015C000BBEC0CF00001C52BC82BA4D7C5C003F1A0
:1015D00045EC0CF0C6C003F1F0EC0DF0C5C003F112
:1015E000EEEC0CF0FF0E0001CA6FCB6B0FD0CAC03F
:1015F000C9F0CAC003F1BBEC0CF012D0CBC0C9F0EB
:10160000CBC003F1BBEC0CF00BD00AD00001C751EA
:10161000000AEDE0C751010AF1E0C751020AF5E006
:10162000120015C0E9FF16C0EAFFEECF00F021500E
:10163000001215C0E1FF16C0E2FF00C0E6FF15C0B2
:10164000E9FF16C0EAFFEECF00F01850001615C0F3
:10165000E1FF16C0E2FF00C0E6FF15C0E9FF16C0BB
:10166000EAFFEECF00F02250001215C0E1FF16C0D5
:10167000E2FF00C0E6FF120E1B24016E000E1C20CC
:10168000026E01C023F002C024F001C0E9FF02C0D5
:10169000EAFFEECF00F02550001201C0E1FF02C0CA
:1016A000E2FF00C0E6FF15C0E9FF16C0EAFFEECF7B
:1016B00000F01750001215C0E1FF16C0E2FF00C095
:1016C000E6FF1BC0E9FF1CC0EAFFEECF03F115C027
:1016D000E9FF16C0EAFFEECF00F01850001615C063
:1016E000E1FF16C0E2FF00C0E6FF15C0E9FF16C02B
:1016F000EAFFEECF00F01A50001615C0E1FF16C049
:10170000E2FF00C0E6FF23C0E9FF24C0EAFFEECFFE
:1017100000F02650001623C0E1FF24C0E2FF00C005
:10172000E6FF03C100F012000001BD6BBE6BBF6B92
:10173000BD5107085BE30101036B45EC0CF0BDC034
:1017400003F1F0EC0DF00101036BEEEC0CF0000185
:10175000BC6BBC513F081AE3BE51B925006EBF51A6
:10176000BA21016E000EBB21026E000E00C0F6FF12
:1017700001C0F7FF02C0F8FF0900F5CF03F1BBEC91
:101780000CF00001BE4BBF2BBC2BE3D7400E010178
:10179000036F45EC0CF0BDC003F1F0EC0DF0400E12
:1017A0000101036FEEEC0CF0400E0001BC6FBC5168
:1017B0007F081AE3BE51B925006EBF51BA21016EF0
:1017C000000EBB21026E000E00C0F6FF01C0F7FF45
:1017D00002C0F8FF0900F5CF03F1BBEC0CF00001EB
:1017E000BE4BBF2BBC2BE3D7BD2BA2D7120015C01D
:1017F000E9FF16C0EAFFEECF00F01F5000162050A0
:10180000001215C0E1FF16C0E2FF00C0E6FF0001B4
:10181000BB6BBB51070812E3BBC003F1F0EC0DF04A
:101820000001BA6BBA513F0807E3B9C003F1BBEC42
:101830000CF00001BA2BF6D7BB2BEBD715C0E9FF94
:1018400016C0EAFFEECF00F01E5000161D50001229
:1018500015C0E1FF16C0E2FF00C0E6FFBB6BBB5145
:10186000070812E3BBC003F1F0EC0DF00001BA6B06
:10187000BA513F0807E3B9C003F1BBEC0CF000011B
:10188000BA2BF6D7BB2BEBD712007F0E0101031545
:10189000016E01C003F101AC1DD015C0E9FF16C0F7
:1018A000EAFFEECF00F01D50001215C0E1FF16C098
:1018B000E2FF00C0E6FF15C0E9FF16C0EAFFEECF69
:1018C00000F01E50001615C0E1FF16C0E2FF00C078
:1018D000E6FF1CD015C0E9FF16C0EAFFEECF00F00E
:1018E0001F50001615C0E1FF16C0E2FF00C0E6FF62
:1018F00015C0E9FF16C0EAFFEECF00F0205000123D
:1019000015C0E1FF16C0E2FF00C0E6FF12000001B3
:1019100000500402F4CF09F0F3CF08F001500502A3
:10192000F4CF0BF0F3CF0AF000500502F350092674
:10193000F4500A22E86A0B2201500402F3500926EF
:10194000F4500A22E86A0B2205AEABEF0CF000500F
:101950000A5C01500B5801AEB2EF0CF004500A5C67
:1019600005500B5808C000F009C001F00AC002F091
:101970000BC003F0120015C0E9FF16C0EAFFEECF5E
:1019800000F01850001615C0E1FF16C0E2FF00C0BD
:10199000E6FF15C0E9FF16C0EAFFEECF00F02150C8
:1019A000001215C0E1FF16C0E2FF00C0E6FF15C03F
:1019B000E9FF16C0EAFFEECF00F01A50001615C07E
:1019C000E1FF16C0E2FF00C0E6FF1BC0E1FF1CC044
:1019D000E2FF03C1E6FFB3EC0DF012007F0E010140
:1019E000031715C0E9FF16C0EAFFEECF00F019504B
:1019F000001615C0E1FF16C0E2FF00C0E6FF15C0EB
:101A0000E9FF16C0EAFFEECF00F01A50001615C02D
:101A1000E1FF16C0E2FF00C0E6FFBF0E0315006E37
:101A200000C003F1008C00C003F11BC0E1FF1CC02B
:101A3000E2FF00C0E6FFB3EC0DF0120000010B6AFC
:101A40000A6A096A00500402F4CF09F0F3CF08F0E3
:101A500001500502F4CF0BF0F3CF0AF0005005025D
:101A6000F3500926F4500A22E86A0B2201500402BE
:101A7000F3500926F4500A22E86A0B2208C000F04D
:101A800009C001F00AC002F00BC003F01200BE0E44
:101A90000001C26F000EC36FB9C0C4F0BAC0C5F078
:101AA000BBC0C6F0BCC0C7F0BDC0C8F0C20EC96F95
:101AB000000ECA6F04EC00F000C0C0F001C0C1F01D
:101AC00000500001B925E16E0150BA21E26EE66ACC
:101AD000C0C000F0C1C001F012000001BE6BBE51D9
:101AE000B925E96E000EBA21EA6EEECF00F0005281
:101AF00018E0BE51B925E96E000EBA21EA6EEECFAC
:101B0000C4F0BBC0C5F0BCC0C6F0BDC0C7F06EEC31
:101B10000AF02950010F006E00500001BB27BE2BB8
:101B2000DED71200150E0C6EFF0E0B6EFF0E0A6E46
:101B30000C2E01D007D00B2E01D003D00A2EFED7D9
:101B4000FAD7F6D7660E0B6EFF0E0A6E0B2E01D07B
:101B500003D00A2EFED7FAD7120E0A6E0A2EFED72F
:101B600000000000120015C0E9FF16C0EAFFEECF2A
:101B700000F01750001215C0E1FF16C0E2FF00C0D0
:101B8000E6FF29EC0EF015C0E9FF16C0EAFFEECF24
:101B900000F01850001615C0E1FF16C0E2FF00C0AB
:101BA000E6FF12000001086A096A100E0C6E01348B
:101BB000083609360450085E0550D8A0053C095E79
:101BC000D8B0EAEF0DF0045008260550D8B0053C17
:101BD0000926D890003601360C2ED7EF0DF01200F2
:101BE00015C0E9FF16C0EAFFEECF00F0195000164D
:101BF0001A50001615C0E1FF16C0E2FF00C0E6FF54
:101C0000B80E01010311006E1BC0E1FF1CC0E2FF12
:101C100000C0E6FFB3EC0DF01200B9C02AF0BAC064
:101C20002BF0BBC02CF0BEC027F0BFC028F0BCC05A
:101C300029F0BDC02FF0120001010351390807E35C
:101C4000300E035D04E3010E006E28EF0EF0006A13
:101C50001200060E0A6E0A2EFED7000012001200B5
:101C600001000A006400E8031027010010000001D1
:101C70000010010008004000000200100080303118
:101C8000323334353637383941424344454600FF14
:101C900030313233343536373839616263646566E2
:101CA00000FF7CA2928A7C0084FE800084C2A29203
:101CB0008C42828A9662302824FE204E8A8A8A725A
:101CC000789492926002E2120A066C9292926C0CE4
:101CD0009292523C00000000004020100804FEFEDA
:101CE0007C38100000040000000005000000000621
:101CF00000000000070000FC222222FCFE929292CB
:101D00006C7C82828244FE82824438FE929292826D
:101D1000FE121212027C828292F4FE101010FE005B
:101D200082FE82004080827E02FE10284482FE8075
:101D3000808080FE041804FEFE081020FE7C828253
:101D4000827CFE1212120C7C82A242BCFE12325223
:101D50008C8C929292620202FE02027E8080807ED1
:101D60003E4080403E7E8070807EC6281028C60E91
:101D700010E0100EC2A2928A86FF0000000000F060
:101D8000F0F070707070F0F0E0C00000F0F0F00063
:101D90000000C0E0E0F070707070E0E0C080000013
:101DA00000000000000000F0F0F070707070F0F0C3
:101DB000E0C0000000000000000000000000000083
:101DC0000000000000000000003030300000000083
:101DD0000000000000000000000000000000000003
:101DE00000000000000080C0E000000000000000D3
:101DF000000000000000000000000000000000FFE4
:101E0000FFFF1C1C1C1C1E1F0F070000FFFFFF0014
:101E1000007FFFFFC1800000000080C1C180000082
:101E200000000000000000FFFFFF1C1C1C1C1E1F08
:101E30000F070000FFFFFF0603030300F8FEFE0785
:101E400003030307FEFEF80000FFFFFF0000F8FE9B
:101E5000FE37333337BEBEB80000F8FEFE0703037B
:101E6000078E8E880003FFFFFF03030000000000C1
:101E7000000000000000000000000000000000075B
:101E800007070000000000E0E0E0E0E0E7E7E7E04F
:101E9000C0800103030707070707030301000000D1
:101EA000000000000000000707070000000000001D
:101EB0000000000007070700000000000003E3E740
:101EC000E606060703030060607F7F3F0000000313
:101ED00003070606070303000000000303070606C6
:101EE00007030300000003070706060000000000C8
:101EF00000000000000000000000000000000000E2
:101F000000000000000000FFFFFF38383838383F7D
:101F1000FFE7C00000F0FCFC0E0606060EFCFCF01D
:101F2000000088CCE666663636FEFCF80000FEFE51
:101F3000FE0C06060600F0FCFC0E0606060CFFFF73
:101F4000FF00000000000000000000000000000092
:101F50000000000000000000000000000000000081
:101F60000000000000000000000000000000000071
:101F70000000000000000000000000000000000061
:101F8000000000000000000F0F0F0E0E0E0E0E0ED0
:101F90000F070300000107070E0C0C0C0E070701CA
:101FA000000003070F0C0C0C06070F0F08000F0FA3
:101FB0000F00000000000107070E0C0C0C060F0FAD
:101FC0000F00000000000000000000000000000002
:101FD0000000000000000000000000000000000001
:101FE00000000000000000000000000000000000F1
:101FF00000000000000000000000000000000000E1
:1020000000E0E0E0E0E0E0E0E0E0C0800000E0E0F0
:10201000E000000080C0C0E0E0E0E0E0C0C0000000
:102020000000008080C0E0E00000000080C0E060B0
:102030006060E0C0800000E0E0E0E0E0E0E0E0E0E0
:10204000E00000000000C0E0E0E0000000000080D0
:10205000E0E06060606000000080C0E0606060E020
:10206000C080000000C0C0E060E0C0C00000000010
:102070000000000000000000000000000000000060
:1020800000FFFFFF383838383D3F1F0F0000FFFFCB
:10209000FF00007EFFFF810000000081C3C38100BC
:1020A0000000070301FFFFFF00000000C3E7FF3C43
:1020B000183CFFE7C30000FFFFFF1C1C1C1C1C1C7E
:1020C0000000E0F0DCCFC3FFFFFFC0C000008C8F3A
:1020D0008F07060EFEFCF80000C3E7FF3C183CFF2C
:1020E000E7C30000FFFFFF000000FFFFFF0000004C
:1020F00000000000000000000000000000000000E0
:1021000000070707000000000000000000000707AC
:102110000700000001030307070707070303000088
:102120000000000000070707000000000103070689
:102130000606070301000007070700000000000073
:102140000000000000000007070700000000010376
:102150000707060707030000000103070606060736
:10216000030100000003030706070303000000004B
:10217000000000000000000000000000000000005F
:102180000000000000000000C0E0E0F0707070F09F
:10219000F0E0C080000080C0E0F0F0707070F0F0FF
:1021A000E0C080000000000000000000000080E0AF
:1021B000E0F0707070F0E0E0800000000080E0E08F
:1021C000F0707070F0E0E08000000000000000801F
:1021D000C0E0F0F0F00000000000000080C0E0E08F
:1021E000F0F0F0F0F0F0F0E0E0C08000000000005F
:1021F00000000000000000000000000000000000DF
:1022000000000000000000030303030080C0E0F0B2
:10221000FF7F3F0F0000078FDFFFF8707070F8FF3F
:10222000DF8F0700000000000000000000FEFFFF3D
:10223000FF0100000001FFFFFFFE0000FEFFFFFFA7
:102240000100000001FFFFFFFE0000001E0F0F074E
:1022500003FFFFFFFF0000000000FCFFFFFF07017E
:102260000100000000000103070703020000000056
:10227000000000000000000000000000000000005E
:1022800000000000000000C0F0FCFEFFEFE7E3E10B
:10229000E0E0E0E000001F3F7F7FF0E0E0E0F07F63
:1022A0007F3F1F000000F0F0F0F0000000071F7FEC
:1022B0007FF8E0E0E0F87F7F1F070000071F7F7FC7
:1022C000F8E0E0E0F87F7F1F07000000000000005A
:1022D00000FFFFFFFF0000000000030F1F3F7E789C
:1022E000F8F0F0F0F0F8F87E7F3F1E0600000000E6
:1022F00000000000000000000000000000000000DE
:102300000000F000000000000000000000000000DD
:1023100000000000000000000000000000000000BD
:1023200000000000000000000000000000000000AD
:10233000000000000000000000000000000000009D
:10234000000000000000000000000000000000008D
:10235000000000000000000000000000000000007D
:10236000000000000000000000000000000000006D
:10237000000000000000000000000000000000005D
:102380000000FF00000000000000000000808080CE
:10239000808080808080C07010101010101010108D
:1023A0001030202020202020E080808080808080CD
:1023B000800000000000000000000000000000009D
:1023C000000000000000000000000000000000000D
:1023D00000000000000000000000000000000000FD
:1023E00000000000000000000000000000000000ED
:1023F00000000000000000000000000000000000DD
:102400000000FF04040404040404040603000000A4
:1024100000000000000000000000000000000000BC
:1024200000000000000000000000000000000000AC
:102430000101020202020202020202060404040472
:1024400004040404040404040404040404041C3008
:10245000202020202020202020202020202020207C
:102460002020202020201008080808080808080854
:102470000808080000000000000000000000000044
:102480000000FF000000000000000000000000004D
:10249000000000000000000000000000000000003C
:1024A000000000000000000000000000000000002C
:1024B000000000000000000000000000000000001C
:1024C000000000000000000000000000000000000C
:1024D00000000000000000000000000000000000FC
:1024E00000000000000000000000000000000000EC
:1024F00000000000000000000000000000000000DC
:1025000000000702020202020202020202020202AA
:10251000020202020202020202020202020202029B
:10252000020202020202020202020202020202028B
:10253000020202020202020202020202020202027B
:10254000020202020202020202020202020202026B
:10255000020202020202020202020202020202025B
:10256000020202020202020202020202020202024B
:102570000202020200000000000000000000000053
:10258000004F00000007000700147F147F14242A66
:102590007F2A12231308646236495522200005035E
:1025A0000000001C2241000041221C0014083E08CB
:1025B0001408083E08085030000000080808080801
:1025C000006060000020100804023E5149453E00B2
:1025D000427F400042615149462141454B31181428
:1025E000127F1027454545393C4A49493001710958
:1025F00005033649494936064949291E0036360041
:10260000000056360000081422410014141414145B
:10261000004122140802015109063E415D551E7E0B
:102620001111117E7F494949363E414141227F4186
:1026300041221C7F494949417F090909013E41491D
:10264000497A7F0808087F00417F41002040413FD0
:10265000017F081422417F404040407F020C027FEE
:102660007F0408107F3E4141413E7F090909063E33
:102670004151215E7F091929462649494932010104
:102680007F01013F4040403F1F2040201F3F403816
:10269000403F6314081463070870080761514945F7
:1026A00043007F41410002040810200041417F00A7
:1026B00004020102044040404040000003050020A5
:1026C000545454787F44444438384444444438444F
:1026D00044447F385454541804047E050508545467
:1026E000543C7F0804047800447D40002040443D71
:1026F000007F1028440000417F40007C047C047867
:102700007C0804047838444444387C1414140808C1
:102710001414147C7C080404004854545424040405
:102720003F44443C4040207C1C2040201C3C403026
:10273000403C44281028440C5050503C4464544CB5
:10274000440836414100000077000000414136084E
:1027500008082A1C08081C2A0808FFFFFFFFFF06BC
:1027600009090600444154413D25584800FFFFFF38
:020000040030CA
:0E000000FFFAFFFEFFFFFBFFFFFFFFFFFFFF0A
:00000001FF
